:1000000000308A0004280000840183131F30830518
:10001000193083169900A63098009030831298000A
:1000200083161F149F141F159F1107309C00FF306B
:100030008312A00083161F109F141F159F151F13F6
:1000400083121F139F1383169F1383121F1483168B
:10005000091283129412A0122008831687008312BB
:1000600020162008831687008312A011200883160B
:100070008700013083129400003083169400010839
:10008000C73908388100831290010030F800043825
:100090009200FF30831692008312201120088316ED
:1000A0008700831207110C309700950107308316E3
:1000B0009C00050885000330F700F70B5D281C083D
:1000C00083120D1383169D0183121F151F196628B5
:0C00D0001E08A1002108950065286300AF
:02400E0039393E
:00000001FF
